:1000000002285D3095FD2095FD2222020B22E70992
:10001000F608DFFA8046E709F208DFFA803E8882B8
:100020008C83E709F0A3DFFA8032E309F608DFFAF0
:100030008078E309F208DFFA807088828C83E30914
:10004000F0A3DFFA806489828A83E0A3F608DFFAEE
:10005000805889828A83E0A3F208DFFA804C80D23C
:1000600080FA80C680D4806980F28033801080A6B8
:1000700080EA809A80A880DA80E280CA8033898210
:100080008A83ECFAE493A3C8C582C8CCC583CCF0BC
:10009000A3C8C582C8CCC583CCDFE9DEE7800D8963
:1000A000828A83E493A3F608DFF9ECFAA9F0EDFB6A
:1000B0002289828A83ECFAE0A3C8C582C8CCC583B2
:1000C000CCF0A3C8C582C8CCC583CCDFEADEE8800B
:1000D000DB89828A83E493A3F208DFF980CC88F07D
:1000E000EF60010E4E60C388F0ED2402B4040050AE
:1000F000B9F582EB2402B4040050AF2323458223D8
:1001000090005E73BB010689828A83E0225002E779
:1001100022BBFE02E32289828A83E49322BB010C84
:10012000E58229F582E5833AF583E0225006E92548
:1001300082F8E622BBFE06E92582F8E222E5822962
:10014000F582E5833AF583E49322BB010689828A2E
:1001500083F0225002F722BBFE01F322F8BB010D0F
:10016000E58229F582E5833AF583E8F0225006E935
:100170002582C8F622BBFE05E92582C8F222EF8D52
:10018000F0A4A8F0CF8CF0A428CE8DF0A42EFE22EF
:10019000C5F0F8A3E028F0C5F0F8E58215827002FA
:1001A0001583E038F022A3F8E0C5F025F0F0E582F1
:1001B000158270021583E0C838F0E822BB010A8975
:1001C000828A83E0F5F0A3E022500687F009E71960
:1001D00022BBFE07E3F5F009E3192289828A83E452
:1001E00093F5F074019322BB0110E58229F582E5B5
:1001F000833AF583E0F5F0A3E0225009E92582F87F
:1002000086F008E622BBFE0AE92582F8E2F5F0084E
:10021000E222E5832AF583E993F5F0A3E99322F836
:10022000BB0111E58229F582E5833AF583E8F0E523
:10023000F0A3F0225009E92582C8F608A6F022BBF7
:10024000FE09E92582C8F2E5F008F222E88FF0A461
:10025000CC8BF0A42CFCE98EF0A42CFC8AF0EDA44D
:100260002CFCEA8EF0A4CDA8F08BF0A42DCC382580
:10027000F0FDE98FF0A42CCD35F0FCEB8EF0A4FE60
:10028000A9F0EB8FF0A4CFC5F02ECD39FEE43CFCF5
:10029000EAA42DCE35F0FDE43CFC2275F008758211
:1002A00000EF2FFFEE33FECD33CDCC33CCC5823300
:1002B000C5829BED9AEC99E58298400CF582EE9B05
:1002C000FEED9AFDEC99FC0FD5F0D6E4CEFBE4CD23
:1002D000FAE4CCF9A88222B800C1B90059BA002DBD
:1002E000EC8BF084CFCECDFCE5F0CBF97818EF2F76
:1002F000FFEE33FEED33FDEC33FCEB33FB10D703A5
:10030000994004EB99FB0FD8E5E4F9FA227818EF4D
:100310002FFFEE33FEED33FDEC33FCC933C910D7AC
:10032000059BE99A4007EC9BFCE99AF90FD8E0E4B9
:10033000C9FAE4CCFB2275F010EF2FFFEE33FEED8F
:1003400033FDCC33CCC833C810D7079BEC9AE8995F
:10035000400AED9BFDEC9AFCE899F80FD5F0DAE441
:10036000CDFBE4CCFAE4C8F922EB9FF5F0EA9E421B
:10037000F0E99D42F0EC6480C864809845F022EB7F
:100380009FF5F0EA9E42F0E99D42F0E89C45F0229C
:10039000E86010ECA2E713FCED13FDEE13FEEF1383
:1003A000FFD8F022E8600FEFC333FFEE33FEED33EA
:1003B000FDEC33FCD8F122BB010789828A83020558
:1003C000565005E9F802054ABBFE05E9F802056248
:1003D00089828A8302056EBB010DE58229F582E5DB
:1003E000833AF5830205565007E92582F802054A4B
:1003F000BBFE07E92582F8020562E58229F582E560
:10040000833AF58302056EBB010789828A83020461
:100410009A5005E9F802057EBBFE05E9F802058A57
:1004200022BB010DE58229F582E5833AF5830204BA
:100430009A5007E92582F802057EBBFE07E925826E
:10044000F802058A227401FF3395E0FEFDFC0808DE
:1004500008E62FFFF618E63EFEF618E63DFDF61814
:10046000E63CFCF6227401FF3395E0FEFDFCA3A3FD
:10047000A3E02FFFF0E582158270021583E03EFEB7
:10048000F0E582158270021583E03DFDF0E58215EE
:100490008270021583E03CFCF022ECF0A3EDF0A3A7
:1004A000EEF0A3EFF022A8828583F0D083D08212F1
:1004B00004BD1204BD1204BD1204BDE473E493A391
:1004C000C583C5F0C583C8C582C8F0A3C583C5F080
:1004D000C583C8C582C822BB010789828A830204FA
:1004E000A65005E9F8020596BBFE05E9F80205AF3E
:1004F00022D083D082F8E4937012740193700DA31C
:10050000A393F8740193F5828883E473740293B51E
:10051000F0067403936860E9A3A3A3A380D8EF4E09
:100520006012EF60010EEDBB010B89828A83F0A39C
:10053000DFFCDEFA2289F05007F709DFFCA9F02280
:10054000BBFEFCF309DFFCA9F022E6FC08E6FD088F
:10055000E6FE08E6FF22E0FCA3E0FDA3E0FEA3E048
:10056000FF22E2FC08E2FD08E2FE08E2FF22E4933B
:10057000FC740193FD740293FE740393FF22ECF666
:1005800008EDF608EEF608EFF622ECF208EDF208B8
:10059000EEF208EFF222D083D082E493F6087401E1
:1005A00093F608740293F608740393F6740473D0F8
:1005B00083D082E493F208740193F208740293F2F8
:1005C00008740393F27404739001A7E0900098F00C
:1005D0007F011240F4900098E09001A7F012326978
:1005E000900091EEF0A3EFF0900091E0FEA3E0FF09
:1005F00064624E6020900098E09001A7F0BEFF0872
:10060000BFFF057EFF7FFF22123269900091EEF05E
:10061000A3EFF080D39001A77401F0E4F5289000D7
:1006200092E02528F528123269900091EEF0A3EFB0
:10063000F064424E70B2E02528F52812326990002D
:1006400091EEF0A3EFF064134E709DE02528F5289D
:10065000123269900091EEF0A3EFF0C39461EE6462
:100660008094804083900091E0FEA3E0FFD3947ECD
:10067000EE6480948040030205E8E02528F528A375
:10068000EEF0A3EFF0E0FF1223B7900091EEF0A39D
:10069000EFF0BEFF10BFFF0D900098E09001A7F0B3
:1006A0007EFF7FFF22900091E07002A3E0600AE4E9
:1006B000900091F0A3F00205D5900093E0FEA3E036
:1006C000FFEE6003020B04EF249FB41B0040030203
:1006D0000B049006D9F828287302072A020735026E
:1006E00007400207950207B10207D402081C02085E
:1006F000640208A20208BE0208DA02090F02091FFA
:1007000002092502094302095602097702098702F4
:1007100009AD0209C00208C9020A1E020A2C020A17
:1007200032020A43020A7A020ADF900094E0FF12C2
:100730003DDB020B0B900094E0FF123DDB020B0B44
:100740009000F27401F0A37400F0A37401F0F9A317
:100750007401F0A37400F0A3E9F07B017A007949F9
:10076000E4FD1214BA90004AE0FD7C00A3E0FB7A9D
:1007700000A3E0FF9000A8E4F0A3EFF07FF31234B1
:10078000CF7B017A007901121333900094E0FF12BD
:100790003DDB020B0B7B017A0079011219F190000D
:1007A00094E0FF7B017A0079017D07123922020B68
:1007B0000B900001E0FFC39401500E123AF190003B
:1007C00094E0FF123DDB020B0B900094E0FF123D22
:1007D000FD020B0B900002E0FEA3E07806C333CECF
:1007E00033CED8F9FDAC067B017A0079499000A59B
:1007F0007440F0900001E0FF122BEFEF70139000B7
:1008000094E0FF7B017A0079497D40123922020B86
:100810000B900094E0FF123DFD020B0B900002E0F4
:10082000FEA3E07806C333CE33CED8F9FDAC0690F4
:10083000009DECF0A3EDF07B017A0079049000A517
:100840007440F0900001E0FF122AF9EF700B900065
:1008500094E0FF123DDB020B0B900094E0FF123D91
:10086000FD020B0B900001E0FFC394015010123801
:10087000D9AD07900094E0FF123E62020B0B90008E
:1008800001E0B4FF127FFF1238D9AD07900094E069
:10089000FF123E62020B0B900094E0FF123DFD023E
:1008A0000B0B12261E90009912049A900094E0FF00
:1008B0007B017A0079997D04123922020B0B90009A
:1008C00001E0FF122C64020B0B900001E0FF7B01A2
:1008D0007A007905122CD6020B0B900001E09000F3
:1008E00097F0601DE0B4FF0512366F8017900097F7
:1008F000E0FF14F0EF600D122FC8EF640160EE808E
:1009000003123F1B900094E0FF123DDB020B0B90A3
:100910000094E0FF123DDB7F011240F4124195127A
:100920002311020B0BE4FF123375EF600B90009460
:10093000E0FF123DFD020B0B900094E0FF123DDB47
:10094000020B0B900094E0FF7B017A01794C7D0C47
:10095000123922020B0B784C7C017D017B017A005D
:1009600079017E007F0C1200DE123EDF900094E0E1
:10097000FF123DDB020B0B900094E0FF900000E0C3
:10098000FD123E62020B0B900001E01424FD5003A7
:10099000020B0BE4900095F0A3F0900094E0FF7B35
:1009A000017A0079957D02123922020B0B90009496
:1009B000E0FF123DDB900001E0FF122DB8020B0BAF
:1009C000900094E0FF123DDB900001E0FF122DB893
:1009D000121E66EF3395E0FE900095F0A3EFF064F1
:1009E0002B4E600E121E66EF3395E0900095F0A33B
:1009F000EFF0900095E07004A3E0642B7018900075
:100A000094E0FF123DDB900094E0FF123DDB90008C
:100A100094E0FF123DDBE4FF122DB8020B0B9000B7
:100A200094E0FF123DDB12418B020B0B12203B02C4
:100A30000B0B900001E0FF7B017A0079021221B7D5
:100A4000020B0B900001E0B4FF0DD200900094E087
:100A5000FF123DDB020B0B900001E0FFC39420501E
:100A60000E121161900094E0FF123DDB020B0B901F
:100A70000094E0FF123DFD020B0B900001E0603F8F
:100A8000046003020B0B900002E0F47028A3E0F472
:100A90007023A3E0F4701EA3E0B4FF19A3E0B4FF39
:100AA00014A3E0B4FF0FA3E0B4FF0A900094E0FFAA
:100AB000123DDB8056900094E0FF123DFD804C7BA0
:100AC000017A007902124118EF700A900094E0FF59
:100AD000123DDB8036900094E0FF123DFD802C1229
:100AE000314E900049EEF0A3EFF01230ED90004B44
:100AF000EFF0900094E0FF7B017A0079497D0312CA
:100B000039228007E4900093F0A3F0900093E0FE78
:100B1000A3E0FF4E70030205D5900098E09001A776
:100B2000F022C0E0C0F0C083C082C0D075D008C23F
:100B30008C758A3E758C5DD28C05179001A6E0609D
:100B40000214F0A2B5B392B5300516E517541C7027
:100B500010E517A2E192A492A392A292A192A08082
:100B60003DE517A2E39208301804A2088002A222F1
:100B700092A0301704A2088002A22192A13016048C
:100B8000A2088002A21F92A2301504A2088002A22D
:100B90001E92A3301404A2088002A21D92A4301257
:100BA00003020D55E51225E0FFE51133FEA287E4AF
:100BB00033FDEEF511EF4DF51230950620100312BE
:100BC000418BA2959210AF1CAE1BAD1AAC19EC4D27
:100BD0004E4F6036A290B3301901B3401D7819749E
:100BE000FF120447EC4D4E4F7044301909D224D205
:100BF000257518FA8038D2098034751C00751B00E1
:100C0000751A00751900B2198024A290B330190129
:100C1000B3501B301908E47F20FEFDFC8006E47F02
:100C200003FEFDFC8F1C8E1B8D1A8C19B219201926
:100C3000033025067E007F0180047E007F00EE4F9A
:100C400024FFB3921DC214E517541F14602F1460C3
:100C500076147003020D4624036003020D55E51857
:100C60007003020D551518E518600BE517A2E59203
:100C7000A592A7020D55D2A7D2A5020D5520133E6D
:100C80000516E51670020515D39457E51594024034
:100C900006751500751600E5168515F01204F10CA1
:100CA000B600000CBA000F0CAF024F00000CC030B1
:100CB000810EC281800AD21B8006D2818002D2209E
:100CC000A220921F020D55201173E5124511600EEE
:100CD000E5122401FFE435114F6003D38001C39274
:100CE0000E30040B200E08751303751484800C203D
:100CF0000409300E0675130175142CE514451360B4
:100D000036E5141514700215131445137029A20644
:100D1000300E01B3401FA20EB39206A206E433FFC9
:100D2000E51870047E0180027E00EE5F6009751890
:100D3000FAD20A8002D20DA20E92048002C206A24A
:100D400006B39221800FE51730E502D201051FE5B9
:100D50001F7002D203D0D0D082D083D0F0D0E03246
:100D6000123B9C1218BC9001A77401F012320C9037
:100D70000000EFF0603C24FD601114601514601950
:100D8000240370237F02123D7380277F03123D737B
:100D900080207F04123D738019E4FB7D017F0512E2
:100DA00027CF123F39800B9000007406F07F0A12A3
:100DB0003D73E49000A8F0A3F0FBFA7D01FC7FF105
:100DC0001234CF9001A77402F01240CA300F031200
:100DD0002E947D017FFF1226B0E4FF122DB8300B58
:100DE00024300F21122E94C2A57FF47E011240867A
:100DF000D2A5E49000A8F0A3F0FBFA7D02FC7FF1FD
:100E00001234CFD200200B14200F11E49000A8F070
:100E1000A3F0FBFA7D03FC7FF11234CF1232C43011
:100E20000314C20320020F12320CEF600924FB608E
:100E300005800012419512261E90008912049A9096
:100E40000182E0FCA3E0FDA3E0FEA3E02416FFEE98
:100E500034FCFEED34FFFDEC34FFFC900089E0F83B
:100E6000A3E0F9A3E0FAA3E0FBD312037F400BE475
:100E7000FB7D017F051227CF8047E47F03FEFDFC49
:100E8000900182E0F8A3E0F9A3E0FAA3E0FB1202EC
:100E90004CE47B04FAF9F81202D7900089E0F8A339
:100EA000E0F9A3E0FAA3E0FBD312037F400B7B0140
:100EB000E4FD7F051227CF8008E4FBFD7F051227A4
:100EC000CFA20FB3920B300B18E4FB7D017F02120F
:100ED00027CF9000007401F0123D4D1237AE020D85
:100EE000D9E4FBFD7F021227CFE4900000F0123717
:100EF000AE8014E51EC394205009AF1E1211610587
:100F00001E80F0151EC20074082510F510C3942031
:100F10004003E4F510E5102407FDAF10121F52EF57
:100F2000600312419530012BC201E490008DF00561
:100F30001EE51EC394204003E4F51EE51EC3942065
:100F40005005AF1E12116190008DE004F0E0C394D3
:100F50000340DC7F967E0012408612331D120F6420
:100F6000020DD9227B017A00799F1237FA7B017A30
:100F70000079901219F112261E90009B12049A7BA0
:100F8000017A01797E1231AD7F2A123B6590008E85
:100F9000741BF0FF123E4190008EE02528F528E4F6
:100FA000A3F07B0190009804F0A37400F0A3749B5D
:100FB000F0900098E0FBA3E0FAA3E0F9120104FF2F
:100FC000123E41900098E0FBA3E475F0011201A6E7
:100FD000A9F0FA1201042528F52890008FE004F00A
:100FE000E0C3940440CBE490008FF07B0190009824
:100FF00004F0A37400F0A37490F0900098E0FBA3B9
:10100000E0FAA3E0F9120104FF123E41900098E0DB
:10101000FBA3E475F0011201A6A9F0FA1201042560
:1010200028F52890008FE004F0E0C3940740CBE45B
:1010300090008FF07B0190009804F0A37401F0A35E
:10104000747EF0900098E0FBA3E0FAA3E0F91201AF
:1010500004FF123E41900098E0FBA3E475F00112FA
:1010600001A6A9F0FA1201042528F52890008FE0C6
:1010700004F0E0C3940440CBE490008FF07B019037
:10108000009804F0A37401F0A37482F0900098E03B
:10109000FBA3E0FAA3E0F9120104FF123E41900025
:1010A00098E0FBA3E475F0011201A6A9F0FA120181
:1010B000042528F52890008FE004F0E0C394044054
:1010C000CBE490008FF07B0190009804F0A37400B3
:1010D000F0A374A3F0900098E0FBA3E0FAA3E0F97A
:1010E000120104FF123E41900098E0FBA3E475F06A
:1010F000011201A6A9F0FA1201042528F528900092
:101100008FE004F0E0C3940440CBE490008FF07BC8
:101110000190009804F0A37400F0A3749FF0900075
:1011200098E0FBA3E0FAA3E0F9120104FF123E41AC
:10113000900098E0FBA3E475F0011201A6A9F0FA73
:101140001201042528F52890008FE004F0E0C394F4
:101150000440CBAF28123E4112400F7F011240F4F1
:101160002290009FEFF0123AB39000CBEEF0A3EF85
:10117000F07B017A01795A90009FE0FD7C00123EDD
:10118000C090015AE0FEA3E0FFF47002EEF4700399
:10119000021330EF4E7003021330E49000C2F0905F
:1011A00000C2E0FFC3942140030212909000A0749B
:1011B000FFF07B017A0079CF90009FE0FD9000D78F
:1011C000EFF0123C6B9000D1E0FEA3E0FF4E700305
:1011D000021273EFF47002EEF470030212739000C7
:1011E000CFE0FCA3E0FDF47002ECF4700302127394
:1011F000ED2FFFEC3EFEC3EF9410EE942750747B6E
:10120000017A0079CD9000CFE0A3E0123F56900024
:10121000CDE0FEA3E0FFEE547FFCEF4C7055EEC432
:1012200013131354019000A0F09000D174FFF5F057
:1012300012019045F0603C7B017A0079CD9000CF9F
:10124000E475F001120190ADF0FC123F569000CD14
:10125000E0FEA3E0FFEE547FFCC39000CCE09F9043
:1012600000CBE09C400DEEC413131354019000A07A
:10127000F080B69000A0E0FF9000C2E024A1F582CB
:10128000E43400F583EFF09000C2E004F002119F17
:1012900090015AE0FEA3E0FF7B017A0079A11224BD
:1012A0005AEF60187F1E7E0012408690015AE0FEC1
:1012B000A3E0FF7B017A0079A112245A9000A1E0FB
:1012C000FF9000A0F090009FE0FE245EF582E434E1
:1012D00001F583E06F60569000A0E0FFC364809446
:1012E00080404A745E2EF582E43401F583EFF0EF1E
:1012F000600C9000CD746FF0A374FEF0800A900033
:10130000CD747FF0A374FEF07B017A0079C31219CB
:10131000F190009FE0FF9000D77401F0A37400F0FB
:10132000A374CDF07B017A0079C312177C7F002271
:101330007F012290009FEBF0A3EAF0A3E9F0900078
:101340009FE0FBA3E0FAA3E0F9120104D394634009
:1013500004E412014A90009FE0FBA3E0FAA3E0F945
:1013600090000112011DFFD3940C5006EFC39401AD
:101370005008900001740112015C90000212011DDE
:10138000FFD3941F5006EFC39401500890000274DD
:101390000112015C90000312011DD39417400790C5
:1013A0000003E412015C90000412011DD3943B4041
:1013B00007900004E412015C90000512011DD39413
:1013C0003B4007900005E412015C90000612011DED
:1013D000D394064007900006E412015CE490018E6D
:1013E000F0A3F090009FE0FBA3E0FAA3E0F99000E7
:1013F0000512011DFF1240E0900190EFF090009F58
:10140000E0FBA3E0FAA3E0F990000412011DFF1233
:1014100040E0900191EFF090009FE0FBA3E0FAA381
:10142000E0F990000312011DFF1240E0900192EFDD
:10143000F090009FE0FBA3E0FAA3E0F99000021215
:10144000011DFF1240E090009FE0FBA3E0FAA3E043
:10145000F9120104FEC4333354C04F900193F0904D
:10146000000112011DFF1240E090009FE0FBA3E08D
:10147000FAA3E0F990000612011DFEC43354E04FB8
:10148000900194F09000F77401F0A37401F0A3743C
:101490008EF0E4FB7D077FA0123BD290009FE0F925
:1014A000A3E0FAA3E09000F7C9F0A3EAF0A3E9F003
:1014B0007B3A7D017FA0123BD2229000EEEBF0A39D
:1014C000EAF0A3E9F09000EEE0FBA3E475F001126E
:1014D00001A6A9F0FAED12014A9000F2E0FBA3E0A8
:1014E000FAA3E0F990000212011DFFC313540FFF8D
:1014F00090000112011DFEC454F04FFF9000EEE079
:10150000FBA3E475F0011201A6A9F0FAEF12014A5B
:101510009000F2E0FBA3E0FAA3E0F99000021201D0
:101520001DFFC43333335480FF120104FEC4333330
:1015300054404FFF90000412011D543F4FFF900094
:10154000EEE0FBA3E475F0011201A6A9F0FAEF1298
:10155000014A9000F2E0FBA3E0FAA3E0F990000555
:1015600012011D75F00A84FFC43354E0FF9000039C
:1015700012011D541F4FFF9000EEE0FBA3E475F035
:10158000011201A6A9F0FAEF12014A9000F5E0FB62
:10159000A3E475F0011201A6A9F0FA120104FF906C
:1015A00000EEE0FBA3E475F0011201A6A9F0FAEF4A
:1015B00012014A9000F5E0FBA3E475F0011201A6C8
:1015C000A9F0FA120104FF9000EEE0FBA3E475F02D
:1015D000011201A6A9F0FAEF12014A9000F5E0FB12
:1015E000A3E475F0011201A6A9F0FA120104FF901C
:1015F00000EEE0FBA3E475F0011201A6A9F0FAEFFA
:1016000012014A9000F5E0FBA3E0FAA3E0F9120111
:1016100004FF9000EEE0FBA3E0FAA3E0F9EF120173
:101620004A22124107900107E0FCA3E0FDA3E0FE7F
:10163000A3E0FF780F120390EFE41241079001A39B
:10164000E024F8600B24E86061241E600302176444
:10165000900107E0FCA3E0FDA3E0FEA3E0FF781803
:10166000120390EC4D4E4F6023900107E0FCA3E085
:10167000FDA3E0FEA3E0FF7807120390EF54FEFF06
:10168000E4EF4401FFE4124107021769900107E00B
:10169000FCA3E0FDA3E0FEA3E0FF7807120390EFB8
:1016A00054FEFFE4124107021769900107E0FCA312
:1016B000E0FDA3E0FEA3E0FF7818120390EC4D4E8E
:1016C0004F6053900107E0FCA3E0FDA3E0FEA3E020
:1016D000FF7807120390EF54FCFFE4FEFDFCEF449B
:1016E00002FFE4C004C005C006C007900107E0FC8B
:1016F000A3E0FDA3E0FEA3E0FF7808120390EF54FF
:1017000001FFE4D003D002D001D000EB4FFFEAE9A3
:10171000E81241078053900107E0FCA3E0FDA3E03D
:10172000FEA3E0FF7808120390EF5401FFE4FEFDF2
:10173000FCC004C005C006C007900107E0FCA3E0A0
:10174000FDA3E0FEA3E0FF7807120390EF54FCFF37
:10175000E4D003D002D001D000EF4BFFEAE9E81259
:10176000410780057F01123F39900107E0FCA3E0AB
:10177000FDA3E0FEA3E0FFE4124107229000D3EFB7
:10178000F0A3EBF0A3EAF0A3E9F07B017A0079E2A1
:101790001237FAEF60037F02229000D3E0FDA3E04E
:1017A000F9A3E0FAA3E09000F2C9F0A3EAF0A3E9FC
:1017B000F09000D7E0F9A3E0FAA3E09000F5C9F0BB
:1017C000A3EAF0A3E9F07B017A0079DA1214BA9067
:1017D00000E2E0FCA3E0FDA3E0FEA3E0FF7B017AD2
:1017E0000079DA1238459000E2120465900182E037
:1017F000F8A3E0F9A3E0FAA3E0FBD312037F500AB9
:101800009000E21204A6000000009000E6E0FCA3B5
:10181000E0FDA3E0FEA3E0FF9000E2E0F8A3E0F922
:10182000A3E0FAA3E0FBC312037F60030218B090A9
:1018300000E6E0FCA3E0FDA3E0FEA3E024E8FFEE69
:101840003403FEE43DFDE43CFC9000E612049A9073
:101850000182E0FCA3E0FDA3E0FEA3E0FF9000E630
:10186000E0F8A3E0F9A3E0FAA3E0FBC312037F4092
:101870002E9000E6E0FCA3E0FDA3E0FEA3E0FF90D5
:101880000182E0F8A3E0F9A3E0FAA3E0FBEF9BFFFD
:10189000EE9AFEED99FDEC98FC9000E612049A9009
:1018A00000EAE07002A3E070079000EAF0A304F001
:1018B0007B017A0079E2123B2D7F0022D2127580E3
:1018C000FF7590FF75A0FF75B0FFE4F510D20175AC
:1018D0001EFFF51FD203C207C224C209C21AC20CDE
:1018E000C20AC20DFBFD7F011227CFE40F1227CFE2
:1018F000E40F1227CFE40F1227CFE40F1227CFD225
:10190000A5D2A7751502751644D220D281D21BD25A
:101910000ED204C206E4F513F5147455F511F51250
:10192000A2959210A290B39219C225E4751C08F5F5
:101930001BF51AF519D20BC205FF7F2090015E74CA
:10194000FFF0A3DFFC7F2012409D7F011240F412C4
:101950004139E4FF122DB8D2B77F1E7E00124086B7
:1019600020B73220B71A7F0A7E0012408620B707C0
:101970007F01123F3980F67F0A7E0012408680E3A5
:10198000123DB97FFF123AF1123F1B123A747F3CAD
:101990007E00124086123FDBEF60227FF47E011250
:1019A00040867F03123F397FF47E011240867F0319
:1019B000123F397FE87E03124086123DB91239F298
:1019C000122F65EF24FFFFE434FFFEE4FCFDFBFA79
:1019D0007901F812024CE47B08FAF9F81239AE905A
:1019E000018212049A1241B79001AA7408F0C2123F
:1019F000229000DBEBF0A3EAF0A3E9F07B017A018F
:101A000079909000F67402F07D057FA0122E279049
:101A10000190E09000DEF07B017A0179909000F671
:101A20007402F07D057FA0122E27900190E0FF90B8
:101A300000DEE06F60137B017A0179909000F6740C
:101A400002F07D057FA0122E277B017A0079DE90BF
:101A500000F6743AF07D017FA0122E27900190E0ED
:101A6000547FFF1241589000DBE0FBA3E0FAA3E0B3
:101A7000F9900005EF12015C900191E0547FFF1294
:101A800041589000DBE0FBA3E0FAA3E0F9900004EA
:101A9000EF12015C900192E0543FFF124158900018
:101AA000DBE0FBA3E0FAA3E0F9900003EF12015C96
:101AB000900193E0543FFF1241589000DBE0FBA3FC
:101AC000E0FAA3E0F9900002EF12015C900194E0CB
:101AD000541FFF1241589000DBE0FBA3E0FAA3E0A3
:101AE000F9900001EF12015C900193E0FFC4131321
:101AF0005403FF9000DEE0FE5403B50706EE12012A
:101B00004A8005EE0412014A900194E0FFC4135488
:101B100007FF9000DBE0FBA3E0FAA3E0F9900006EA
:101B2000EF12015C229000DEEEF0A3EFF0A3EDF0E7
:101B3000A3EBF07F011240F4E49001A7F0123269A8
:101B40009000E9EEF0A3EFF09000E9E0FCA3E0FDE7
:101B5000BCFF06BDFF037F0122ED64034C70DE90E5
:101B6000012BF09000EAE0FF90012BE02FF0123201
:101B7000699000E9EEF0FCA3EFF0FD9000DEE0B527
:101B800005C6E4B504C29000EAE0FF90012BE02F07
:101B9000F01232699000E9EEF0A3EFF09000DFE080
:101BA000B507A5E4B506A19000EAE0FF90012BE09F
:101BB0002FF01232699000E9EEF0A3EFF09000E010
:101BC000E06F7001EE70819000EAE0FF90012BE081
:101BD0002FF09000E1E09000E8F09000E2E0F9A33F
:101BE000E0FAA3E0A3C9F0A3EAF0A3E9F09000E8CB
:101BF000E0D39400403B1232699000E9EEF0A3EF8D
:101C0000F0BEFF06BFFF037F01229000EAE0FF90D5
:101C1000012BE02FF09000E5E0FBA3E475F001124A
:101C200001A6A9F0FAEF12014A9000E8E014F08052
:101C3000BC1232699000E9EEF0A3EFF090012BE0C6
:101C40006F7001EE6003021B487F00229000ACEB36
:101C5000F0A3EAF0A3E9F07B017A0079AF1237FA3A
:101C60009000B3E0FCA3E0FDA3E0FEA3E0FF900042
:101C7000AFE0F8A3E0F9A3E0FAA3E0FBD312037FFF
:101C8000406E9000ACE0FBA3E0FAA3E0F91203B7CA
:101C90009000AFE0F8A3E0F9A3E0FAA3E0FBC312E1
:101CA000037F40229000ACE0FBA3E0FAA3E0F9122E
:101CB00003B79000B3E0F8A3E0F9A3E0FAA3E0FBD8
:101CC000D312037F40159000AFE0FCA3E0FDA3E03A
:101CD000FEA3E0FF90018A12049A229000ACE0FB80
:101CE000A3E0FAA3E0F91203B790018A12049A2242
:101CF0009000ACE0FBA3E0FAA3E0F91203B7900078
:101D0000AFE0F8A3E0F9A3E0FAA3E0FBC312037F7E
:101D100050379000ACE0FBA3E0FAA3E0F91203B760
:101D20009000B3E0F8A3E0F9A3E0FAA3E0FBD3123C
:101D3000037F40159000AFE0FCA3E0FDA3E0FEA30D
:101D4000E0FF90018A12049A229000ACE0FBA3E02D
:101D5000FAA3E0F91203B790018A12049A22094308
:101D600000A00954009F0966009E0977009D09891B
:101D7000009C099B009B09AD009A09BF009909D2FC
:101D8000009809E4009709F700960A0A00950A1DD1
:101D900000940A3000930A4300920A5700910A6B9C
:101DA00000900A7F008F0A93008E0AA7008D0ABB5D
:101DB000008C0AD1008B0AE7008A0AFE00890B1406
:101DC00000880B2B00870B4300860B5C00850B758E
:101DD00000840B8E00830BA700820BC100810BDBFC
:101DE00000800BF6007F0C10007E0C2B007D0C4752
:101DF000007C0C64007B0C81007A0C9E00790CBB8B
:101E000000780CDB00770CFB00760D1B00750D3B9A
:101E100000740D5B00730D7D00720D9F00710DC28B
:101E200000700DE4006F0E07006E0E2C006D0E5159
:101E3000006C0E76006B0E9B006A0EC100690EE905
:101E400000680F1100670F3900660F6100650F8988
:101E500000640FB300630FDE0062100900611034EC
:101E60000060105F005F7F011240F49001A77401D1
:101E7000F0E49000A1F0A3F012326990009FEEF020
:101E8000A3EFF064624E602E90009FE0B4FF08A3C1
:101E9000E0B4FF037FFF229000A2E004F070069000
:101EA00000A1E004F0C39000A2E0940A9000A1E039
:101EB0006480948040C290009FE07004A3E064625C
:101EC00060037F2D2212326990009FEEF0A3EFF0A5
:101ED00064424E60037F2D2212326990009FEEF023
:101EE000A3EFF064134E60037F2D2212326990003D
:101EF0009FEEF0A3EFF064744E60037F2D22123248
:101F00006990009FEEF0A3EFF0BEFF06BFFF037FD6
:101F10002D229000A0E0242BFFE43401E49000A3E4
:101F2000F0EFA3F012326990009FEEF0A3EFF0BE45
:101F3000FF06BFFF037F2D229000A3E0FEA3E0FF7A
:101F400090009FE06E7003A3E06F60037F2D227FFF
:101F50002B2290008EEFF0A3EDF0C3942040037489
:101F60001FF07B017A00799A1219F190008EE090AF
:101F70000090F090008FE0FFA3E0FD3395E0FCD3EC
:101F8000ED9F7480F86C9840030220387B017A0141
:101F9000795A123EC090015AE0FEA3E0FFF47002AD
:101FA000EEF4700302202FEF4E700302202F9001F9
:101FB0005AE0FEA3E0FF7B017A007992122108909B
:101FC0000091EFF07051A3E054F0604B900090E06E
:101FD000FF122741900090E0FF9000D77401F0A31A
:101FE0007400F0A37492F07B017A00799A12177C46
:101FF00090015AE0FEA3E0FF7D0112388FEF60AE42
:102000007F0A7E0012408690015AE0FEA3E0FF7D29
:102010000112388FEF7097900091E0600A90009065
:10202000E0FF1224F38008900090E0FF1227419017
:102030000090E004F0021F737F00227B017A007998
:10204000A01237FA7F77123B65E490009FF0752568
:1020500001752601752782AB25AA26A9271201043E
:10206000FF123E41AB250527E527AA26700205266B
:1020700014F91201042528F52890009FE004F0E0EF
:10208000C3940440D2E490009FF0752501752600AA
:102090007527A0AB25AA26A927120104FF123E41ED
:1020A000AB250527E527AA267002052614F912019B
:1020B000042528F52890009FE004F0E0C394044034
:1020C000D2E490009FF07525017526007527A4AB1A
:1020D00025AA26A927120104FF123E41AB25052798
:1020E000E527AA267002052614F91201042528F511
:1020F0002890009FE004F0E0C3940440D2AF28127F
:102100003E4112400F7F2B229000A2EEF0A3EFF091
:10211000A3EBF0A3EAF0A3E9F09000A97403F09018
:1021200000A2E0FEA3E0FFE4FB7D41122A7A9000CA
:10213000A2E0FEA3E0FF9000E27401F0A37400F0BF
:10214000A374A7F07B027D41121B25EF705790000E
:10215000A7E0FF9000A4E0FBA3E475F0011201A644
:10216000A9F0FAEF12014A9000A8E0FF9000A4E065
:10217000FBA3E475F0011201A6A9F0FAEF12014ADF
:102180009000A4E0FBA3E475F0011201A6A9F0FA07
:10219000E412014A9000A4E0FBA3E0FAA3E0F9E412
:1021A00012014AFF229000A9E014F0E0D39400400D
:1021B0000302211F7F012290009FEFF0A3EBF0A309
:1021C000EAF0A3E9F07F78123B6590009FE0FF14EE
:1021D000F0EF700302225C9000B27401F0A374006F
:1021E000F0A374A4F09000A0E0FBA3E0FAA3E0F950
:1021F0001237119000A0E0FBA3E0FAA3E0F912036C
:10220000B7EF2401FFE43EFEE43DFDE43CFC120494
:10221000079000AC7401F0A37400F0A374A4F090D4
:1022200000A37408F09000A3E0609F9000ACE0FB76
:10223000A3E0FAA3E0F9120104FF123E419000ACC2
:10224000E0FBA3E475F0011201A6A9F0FA12010463
:102250002528F5289000A3E014F080C9AF28123E8D
:102260004112400F227B017A0079981237FAEF6011
:10227000037F02227B017A007998122589C007909A
:102280000182E0FCA3E0FDA3E0FEA3E0FF90009844
:10229000E0F8A3E0F9A3E0FAA3E0FBC312037F4058
:1022A000047E0180027E00D0E04EFFC007900182D4
:1022B000E0FCA3E0FDA3E0FEA3E0FF90009CE0F8BB
:1022C000A3E0F9A3E0FAA3E0FBC312037F40047E7E
:1022D0000180027E00D0E04E60037F022212261EA3
:1022E000A804A905AA06AB07900182E0FCA3E0FDC3
:1022F000A3E0FEA3E02416FFEE34FCFEED34FFFD68
:10230000EC34FFFCD312037F40047F0480027F0083
:10231000227F6D123B657F0D123E41740D2528F51D
:10232000287F14123E4174142528F5287F0D123E93
:1023300041740D2528F5287F3E123E41743E252824
:10234000F5287F80123E4174802528F5287F601291
:102350003E4174602528F528E4FF123E417F0112BA
:102360003E4105287F40123E4174402528F5287FD4
:102370000E123E41740E2528F5287F27123E417427
:10238000272528F5287F10123E4174102528F528AE
:102390009001A3E025E0FF123E419001A3E025E07B
:1023A0002528F5287F20123E4174202528F528FF96
:1023B000123E4112400F2290009F7401F0A374005E
:1023C000F0A37401F0EF903F1193FF7E009000A402
:1023D000EEF0A3EFF0D394487480948040037F0123
:1023E000229000A474FFF5F01201A6FED3E5F0944C
:1023F00000EE6480948040361232699000A2EEF0C4
:10240000A3EFF0BEFF08BFFF057EFF7FFF22900015
:10241000A3E02528F528E0FF90009FE0FBA3E475EA
:10242000F0011201A6A9F0FAEF12014A80B31232AC
:10243000699000A2EEF0A3EFF0BEFF08BFFF057E9B
:10244000FF7FFF229000A2E07004A3E065286005F2
:102450007EFF7FFE227E007F00229000D3EEF0A35D
:10246000EFF0A3EBF0A3EAF0A3E9F0201C29900021
:10247000D3E0FEA3E0FFA3E0FBA3E0FAA3E0F912A0
:102480000104FDC3648094804006EDF4FDFB8002EE
:102490007B00E4FD1234799000D6E475F00112015E
:1024A000909000D87401F09000D8E0FDC3942150C2
:1024B0003F9000D5E0FBA3E0FAA3E0F9120104C3CA
:1024C0006480948040229000D3E0FEA3E0FFA3E06C
:1024D000A3E475F0011201A6A9F0FA120104FB129F
:1024E0003479EF60037F01229000D8E004F080B7D8
:1024F0007F0022EFC394205037742C2FF582E434F0
:1025000001F583E07003022588E014F0707A740B03
:102510002FF582E43401F583E0606DE4F0EFFD7C9B
:1025200000E49000A8F0A3F0FBFA7FF21234CF226F
:10253000E49000A2F09000A2E0FFC3942050497400
:102540002C2FF582E43401F583E06034E014F07060
:102550002F740B2FF582E43401F583E060229000A4
:10256000A2E0FF240BF582E43401F583E4F0EFFDF3
:102570007C00E49000A8F0A3F0FBFA7FF21234CFC5
:102580009000A2E004F080AD229000F1EBF0A3EA0D
:10259000F0A3E9F0E4FFA3F0A3F09000F1E0FBA3C7
:1025A000E0FAA3E0F975F002EFA4F58285F083125A
:1025B00001E7FDACF09000F5E02DF09000F4E03C78
:1025C000F00FEFB406D49000F4E07002A3E070477F
:1025D0009000F1E0FBA3E0FAA3E0F91203B7900149
:1025E00082E0F8A3E0F9A3E0FAA3E0FBD312037FB3
:1025F00040259000F1E0FBA3E0FAA3E0F99000048D
:102600001203D7900182E0F8A3E0F9A3E0FAA3E077
:10261000FBD312037F50047F0180027F00227B01E5
:102620007A0079AB1237FA9000ABE0FCA3E0FDA38F
:10263000E0FEA3E0FFA3E0F8A3E0F9A3E0FAA3E043
:10264000FBD312037F40419000ABE0FCA3E0FDA36D
:10265000E0FEA3E0FF900182E0F8A3E0F9A3E0FA36
:10266000A3E02FFFEA3EFEE93DFDE83CFC9000AF11
:10267000E0F8A3E0F9A3E0FAA3E0C3EF9BFFEE9A32
:10268000FEED99FDEC98FC229000AFE0F8A3E0F994
:10269000A3E0FAA3E0FB9000ABE0FCA3E0FDA3E025
:1026A000FEA3E0C39BFFEE9AFEED99FDEC98FC22A1
:1026B00090008EEDF0EFC39420503CE0FE740B2FA1
:1026C000F582E43401F583EEF0EE14600F04701926
:1026D000742C2FF582E43401F583E4F0742C2FF58B
:1026E00082E43401F583740AF0742C2FF582E4340B
:1026F00001F5837405F0227E007F2090008EE0FDBE
:102700007B017A01790B12051E90008EE014601295
:1027100004701E7E007F207D007B017A01792C12DF
:10272000051E7E007F207D0A7B017A01792C12052F
:102730001E7E007F207D057B017A01792C12051E0B
:1027400022EFC394205031742C2FF582E43401F52C
:1027500083740AF0740B2FF582E43401F583E07082
:102760006D04F0EF4480FD7C00E49000A8F0A3F03D
:10277000FBFA7FF21234CF22E49000A2F09000A284
:10278000E0FFC394205047742C2FF582E43401F508
:1027900083740AF0740B2FF582E43401F583E07042
:1027A000259000A2E0FF240BF582E43401F5837448
:1027B00001F0EF4480FD7C00E49000A8F0A3F0FB62
:1027C000FA7FF21234CF9000A2E004F080AF22EF43
:1027D00024FE602614603C14605214606824047067
:1027E0007BED6003B40106ED24FFB3921DEB6004A2
:1027F00064017068EB24FF921422ED6003B40106BB
:10280000ED24FFB3921EEB60046401704FEB24FFD4
:10281000921522ED6003B40106ED24FFB3921FEB85
:10282000600464017036EB24FF921622ED6003B45D
:102830000106ED24FFB39221EB60046401701DEBEF
:1028400024FF921722ED6003B40106ED24FFB3923A
:1028500022EB6003B40105EB24FF921822787FE499
:10286000F6D8FD7581280228A4020D60E493A3F830
:10287000E493A34003F68001F208DFF48029E49397
:10288000A3F85407240CC8C333C4540F4420C8838E
:102890004004F456800146F6DFE4800B0102040890
:1028A000102040809041AEE47E019360BCA3FF54B1
:1028B0003F30E509541FFEE493A360010ECF54C0DE
:1028C00025E060A840B8E493A3FAE493A3F8E49366
:1028D000A3C8C582C8CAC583CAF0A3C8C582C8CA6E
:1028E000C583CADFE9DEE780BE9000ACEBF0A3EA67
:1028F000F0A3E9F07B017A0079AF1237FA9000AFCC
:10290000E0FCA3E0FDA3E0FEA3E0FF900186E0F879
:10291000A3E0F9A3E0FAA3E0FBC312037F700F90DA
:1029200000ACE0FBA3E0FAA3E0F9124174229001AD
:1029300086E0FCA3E0FDA3E0FEA3E0FF9000ACE096
:10294000FBA3E0FAA3E0F9123A3490018612046581
:10295000900182E0F8A3E0F9A3E0FAA3E0FBD31230
:10296000037F500A9001861204A6000000007F0039
:10297000229000ACEBF0A3EAF0A3E9F07B017A002F
:1029800079AF1237FA9000AFE0FCA3E0FDA3E0FEC0
:10299000A3E0FF90018AE0F8A3E0F9A3E0FAA3E046
:1029A000FBC312037F700F9000ACE0FBA3E0FAA31F
:1029B000E0F91241742290018AE0FCA3E0FDA3E05B
:1029C000FEA3E0FF9000ACE0FBA3E0FAA3E0F91265
:1029D0003A3490018A120465900182E0F8A3E0F98C
:1029E000A3E0FAA3E0FBD312037F500A90018A12FE
:1029F00004A6000000007F00224D6F6E61204C692C
:102A0000736120284350522053746172742900204E
:102A1000435052207665722E32302E3133202028DA
:102A20004329526F67657220532E432E2020476F33
:102A3000736369737A65776F2D4D616C626F726B2A
:102A400020202074656C2E2F6661782E20302D3565
:102A500035203237323031323320202068747470A0
:102A60003A2F2F7777772E726F6765722E706C0012
:102A70004D6F6E61204C697361009000DEEEF0A333
:102A8000EFF0A3EDF0A3EBF0E4FF1240F4E49001CB
:102A90002BF07F09123E4190012BE02409F09000B9
:102AA000DEE0FF123E419000DEE0FF90012BE02FC0
:102AB000F09000DFE0FF123E419000DFE0FF900168
:102AC0002BE02FF09000E0E0FF123E419000E0E0AC
:102AD000FF90012BE02FF09000E1E0FF123E4190CB
:102AE00000E1E0FF90012BE02FF0E0FF123E417F7C
:102AF00006123E417E007F002290009FEFF0A3EC83
:102B0000F0A3EDF0A3EBF0A3EAF0A3E9F0EF04707B
:102B100005E490009FF090009FE004F0E0FED39465
:102B200001501B9000A5E0FDC3E49DFD746094007E
:102B3000FCD39000A1E09D9000A0E09C40037FFFAB
:102B400022EE7F00C43333335480FEE4AA069000A3
:102B5000A0E0FEA3E0FFE42FFFEA3EFEE433FDE445
:102B600033FCA3E0FBA3E0FAA3E0F9A3E09000FCB0
:102B7000F0122B777F00229000F512049A9000F952
:102B8000EBF0A3EAF0A3E9F09000F5E0FCA3E0FD90
:102B9000A3E0FEA3E0FF122D489000F5E0FCA3E0C7
:102BA000FDA3E0FEA3E0FF9000FCE0FB900101E448
:102BB000F0A3EBF09000F9E0F9A3E0FAA3E09001B4
:102BC00003C9F0A3EAF0A3E9F01234239000F5E082
:102BD000FCA3E0FDA3E0FEA3E0FF1239699000F53D
:102BE000E0FCA3E0FDA3E0FEA3E0FF123D2622905F
:102BF000009FEFF0A3ECF0A3EDF0A3EBF0A3EAF05D
:102C0000A3E9F0EF047005E490009FF090009FE0CE
:102C100004F0E0FED39401500E9000A1E0940090E7
:102C200000A0E0946040037FFF22EE7F00C43333B6
:102C3000335480FEE4AA069000A0E0FEA3E0FFE487
:102C40002FFFEA3EFEE433FDE433FC9000A5E09064
:102C500000DFF09000A2E0FBA3E0FAA3E0F9123657
:102C60001D7F002290009FEFF0123EFD7F6A123B15
:102C70006590009FE0FF14F0EF60527B017A0079CD
:102C8000A11228E99000A97401F0A37400F0A374C4
:102C9000A1F09000A07408F09000A0E0FF14F0EF05
:102CA00060CF9000A9E0FBA3E0FAA3E0F9120104D1
:102CB000FF123E419000A9E0FBA3E475F001120170
:102CC000A6A9F0FA1201042528F52880CBAF281216
:102CD0003E4112400F2290009FEFF0121C4C7F7576
:102CE000123B6590009FE0FF14F0EF60527B017A89
:102CF0000079A11229719000A97401F0A37400F069
:102D0000A374A1F09000A07408F09000A0E0FF145C
:102D1000F0EF60CF9000A9E0FBA3E0FAA3E0F91286
:102D20000104FF123E419000A9E0FBA3E475F0010D
:102D30001201A6A9F0FA1201042528F52880CBAFCC
:102D400028123E4112400F229000FD12049A90007A
:102D5000FDE0FCA3E0FDA3E0FEA3E0FF7808120382
:102D600090EFFBEEFAE4F9F89001A4E0FEA3E0FF97
:102D7000E4FCFDC3120369603E123FC1C2849000AF
:102D8000FDE0FCA3E0FDA3E0FEA3E0FF900107123D
:102D9000049A7F53121622D2849000FDE0FCA3E037
:102DA000FDA3E0FEA3E0FF7808120390EFEEE490AD
:102DB00001A4EEF0A3EFF02290009FEFF0C3648037
:102DC0009480500E7F06123F397FD07E07124086D6
:102DD00080F290009FE0700204F090009FE0FF906E
:102DE00001A8F03395E0FEFDFCF8F9FAAB07E47FAB
:102DF00034FEFDFC1239AEAD07AC06C3E49DFDE424
:102E00009CFCE4F5C8C2ADC2ACECFFF5CBAE05EE60
:102E1000F5CA8FCDF5CC759853C298D29975C83440
:102E20009001A77402F0229000F3EBF0A3EAF0A364
:102E3000E9F0AC05AD07EC605A124149ED54F0449D
:102E400002FF123F8D9000F6E0FF123F8D124149C4
:102E5000ED54F04403FF123F8D1CEC601C123FA7A1
:102E60009000F3E0FBA3E475F0011201A6A9F0FACB
:102E7000EF12014A12419F80E0123FA79000F3E059
:102E8000FBA3E475F0011201A6A9F0FAEF12014AC2
:102E900012416722E490008EF090008EE0FFC36440
:102EA0008094A050577B017A01795AEFFD3395E069
:102EB000FC123EC090015AE0FEA3E0FF900097EEA6
:102EC000F0A3EFF04E602D900097E0FEA3E0FF7BB3
:102ED000017A00798F122108EF701990008FE0FFBE
:102EE000C4540F600F900097E0FEA3E0FFE4FD12D2
:102EF000388F80D390008EE004F0809D2290019561
:102F0000EBF0A3EAF0A3E9F0A3EDF0A3E0FDC364C6
:102F1000809480404D900198E0702A201C279001F9
:102F200095E0FBA3E0FAA3E0F91201BCFFAEF0C309
:102F3000ED648094804006EDF4FDFB80027B00E4AC
:102F4000FD12347922900195E0FBA3E0FAA3E0F9A9
:102F50001201BCFFAEF0900198E0FDA3E0FB12343B
:102F600079227F012212412990008EEFF0BFFF0EDF
:102F70007F02123F397FE87E0312408680E790008F
:102F80008EE0543824E8601024F060142420701877
:102F90009001A37402F0802A9001A37408F08022AB
:102FA0009001A37420F0801A7F02123F397FF47ED3
:102FB000011240867F02123F397F887E13124086BD
:102FC00080E69001A3E0FF227B017A00799F12370F
:102FD000FA90009FE0FCA3E0FDA3E0FEA3E0FFA3C6
:102FE000E0F8A3E0F9A3E0FAA3E0FBC312037F60DB
:102FF000379000A3120465900182E0F8A3E0F9A3E2
:10300000E0FAA3E0FBD312037F500A9000A312045E
:10301000A600000000E49000A7F0A3F07B017A0076
:10302000799F123B2D7F00227F01229000F4EBF06C
:10303000A3EAF0A3E9F0E4FFA3F0A3F09000F4E02A
:10304000FBA3E0FAA3E0F975F002EFA4F58285F0A6
:10305000831201E7FDACF09000F8E02DF09000F74E
:10306000E03CF00FEFB405D49000F7E0FEA3E0FFE2
:10307000C3E49FFFE49EFE9000F4E0FBA3E0FAA30C
:10308000E0F990000AEE8FF012021F229000F1EB9F
:10309000F0A3EAF0A3E9F09000F1E0FBA3E0FAA3CB
:1030A000E0F91203B7E4FB7A20F9F8D312037F505A
:1030B000129000F1E0FBA3E0FAA3E0F91204D700BC
:1030C0000000009000F1E0FBA3E0FAA3E0F9120396
:1030D000B7900004120421900008E4F5F012021FDA
:1030E0009000041203D790018612049A22AD07AC17
:1030F0000690009F74FFF0A3741DF0A3745EF0E4CB
:10310000A3F090009FE0FBA3E0FAA3E0F91201BC5A
:10311000FFC3ED9FEC95F050089000021201E7FF0D
:10312000229000A0E475F0041201909000A2E00447
:10313000F0E0B442CD90009FE0FBA374FF75F0FC7B
:10314000120190A9F0FA9000041201E7FF22D28642
:10315000A2A49226D2A47F017E00124086C28E5382
:10316000890F438910E4F58BF58DC28FC2AFC2A4DD
:10317000D28E208603308FFAC28ED2AFA22692A4BE
:10318000AF8DEFFEAD8B7C00E42DFFEC3EAD07FC78
:10319000208F09D3ED94FFEC947F40057EFF7FFFE5
:1031A00022AE04AF05ED25E0FFEC33FE22201D0426
:1031B0007F0180027F00301404EF4402FF201E04D0
:1031C000EF4404FF301504EF4408FF201F04EF44D0
:1031D00010FF301604EF4420FF202104EF4440FF8D
:1031E000301704EF4480FFEF12014A2022047E01D1
:1031F00080027E00AF06301804EF4402FF20A704CF
:10320000EF44C0FF900001EF12015C227FFF1238F3
:10321000D9EF60037F02227B017A00798E1219F1C7
:10322000900093E0D3943B5028900092E0943B5060
:1032300020900091E094175018900090E0941F5057
:103240001090008FE0940C500890008EE094634042
:10325000037F0422122265EF24FC6007240270061B
:103260007F03227F05227F00229001A7E0146019CE
:1032700014603124027048123D97EF6007C298AF86
:10328000997E00227EFF7FFF229001A67414F02019
:10329000980B9001A6E070F77EFF7FFF22C298AFE7
:1032A000997E00229001A67478F020980B9001A6D8
:1032B000E070F77EFF7FFF22C298AF997E00227EEA
:1032C000FF7F9B22300913C209E49000A8F0A3F00D
:1032D000FBFA7D06FC7FF11234CF302413C224E4C4
:1032E0009000A8F0A3F0FBFA7D05FC7FF11234CF2B
:1032F000300D13C20DE49000A8F0A3F0FBFA7D0A94
:10330000FC7FF11234CF300A13C20AE49000A8F017
:10331000A3F0FBFA7D09FC7FF11234CF227F30123B
:103320003E1F7F011240F49001A77401F01205C8FE
:10333000EE703FEF249F703A90008E7403F0A374F8
:10334000E8F090008EE0FEA3E0FFF47002EEF4607F
:103350001EEF64624E60189001A77402F01205C857
:1033600090008EEEF0A3EFF07F011240F480D37F47
:1033700001227F002290009FEFF0C3940140037F61
:10338000FF2290009FE0FF1238D9EF60037FFE22FA
:10339000E49000A0F09000A0E0FFD39460502AEFEA
:1033A000FD7C007E00C00790009FE075F080A4FFC8
:1033B0002480FFE435F0CF2DFDEC3FFCD007123C1C
:1033C000FB9000A0E004F080CC7F002290019AEFF7
:1033D000F0A3EDF0A3EBF0A3EAF0A3E9F0E4FF1211
:1033E00040F490019AE0FF6004F599800375993DDF
:1033F0007F0A7E0012408690019BE0FF14F0EF6090
:103400001CA3E0FBA3E475F0011201A6A9F0FA12D7
:103410000104F5997F0A7E0012408680DA7F01124E
:1034200040F4229000FD12049A123FC1C284900021
:10343000FDE0FCA3E0FDA3E0FEA3E0FF9001071286
:10344000049A7F8412162290010174FFF5F0120194
:10345000A645F06019900103E0FBA3E475F00112AA
:1034600001A6A9F0FA120104FF12410780D9D28403
:1034700074FF9001A4F0A3F0229000D9EEF0A3EF26
:10348000F0A3EDF0A3EBF0A37403F09000D9E0FEFD
:10349000A3E0FFA3E0FD25E0FDA3E054014DFB7D8B
:1034A00044122A7A9000D9E0FEA3E0FF9000E2E403
:1034B000F0A3F0A3F0FB7D44121B25EF7002FF2266
:1034C0009000DDE014F0E0D3940050BF7F01229023
:1034D00000A3EFF0A3ECF0A3EDF0A3EAF0A3EBF070
:1034E0007B017A0079AA1219F19000A3E09000B252
:1034F000F09000A5E09000B3F09000A7E09000B439
:10350000F09000A9E09000B5F09000D77401F0A30E
:103510007400F0A374B2F07B017A0079AA7FFF12E5
:10352000177C2290019FEEF0A3EFF0ED54074428A2
:103530009001A2F09001A17403F090019FE0FEA31E
:10354000E0FF9001A2E0FB7D4B122A7A90019FE000
:10355000FEA3E0FF9000E2E4F0A3F0A3F0FB7D4BBC
:10356000121B25EF7002FF229001A1E014F0E0D3BE
:10357000940050C67F01229000E012049A123FC1CD
:10358000C2849000E0E0FCA3E0FDA3E0FEA3E0FF26
:1035900090010712049A7F54121622E4FF12410789
:1035A0009000E474FFF5F01201A645F06019124096
:1035B000B49000E6E0FBA3E475F0011201A6A9F0C7
:1035C000FAEF12014A80D9D284229000A17401F04E
:1035D000A37401F0A3744CF0E4FF90009FF0A3F0FB
:1035E0009000A1E0FBA3E475F0021201A6A9F0FA95
:1035F0001201BCFDACF09000A0E02DF090009FE027
:103600003CF00FEFB406D990009FE0FEA3E0FFC3AB
:10361000E49FFFE49E900158F0A3EFF0229000D8C1
:10362000EBF0A3EAF0A3E9F0A312049A9000DBE028
:10363000FCA3E0FDA3E0FEA3E0FF122D489000DB19
:10364000E0FCA3E0FDA3E0FEA3E0FFA3E0FB90000D
:10365000E4E4F0A3EBF09000D8E0F9A3E0FAA3E0F3
:103660009000E6C9F0A3EAF0A3E9F0123577227BD7
:10367000017A00799F1237FA900186E0FCA3E0FD01
:10368000A3E0FEA3E0FF9000A3E0F8A3E0F9A3E02D
:10369000FAA3E0FBC312037F6007E49000A7F0A346
:1036A000F0900186E0FCA3E0FDA3E0FEA3E0FF9024
:1036B00000A312049A7B017A00799F123B2D7F00B0
:1036C000229000A4EEF0A3EFF0A3EDF0E4FCFD786F
:1036D000081203A4122D48123FC1C2849000A4E036
:1036E000FEA3E0FFE4FCFD78081203A4900107129A
:1036F000049A7F54121622E4FF124107E4FD12409F
:10370000B4EF2DFD9000A6E014F070F2D284AF0566
:10371000229000AFEBF0A3EAF0A3E9F09000AFE055
:10372000FBA3E0FAA3E0F91203B7900182E0F8A34B
:10373000E0F9A3E0FAA3E0FBD312037F401F90005F
:10374000AFE0FBA3E0FAA3E0F91203B79000B2E008
:10375000FBA3E0FAA3E0F9123A347F00227F0522AE
:103760009000907401F0A37401F0A3744CF0E4FF96
:1037700090008EF0A3F0900090E0FBA3E475F002BF
:103780001201A6A9F0FA1201BCFDACF090008FE086
:103790002DF090008EE03CF00FEFB407D990008E32
:1037A000E07002A3E060047F0180027F0022301BF2
:1037B00048C21B123CCB90008EEFF0D2819001AA40
:1037C000E06F601590008EE0FD7C00E49000A8F0B2
:1037D000A3F0FBFA7FF11234CF90008EE0FFB40823
:1037E00003D38001C3922020200A9001AAE0B408EC
:1037F000037518FA9001AAEFF0229000EEEBF0A307
:10380000EAF0A3E9F09000F67420F07D0C7FA0129E
:103810002E279000EEE0FBA3E0FAA3E0F912258941
:10382000EF601F9000EEE0FBA3E0FAA3E0F9123096
:103830008C9000EEE0FBA3E0FAA3E0F9123B2D7FB1
:1038400001227F00229000EE12049A9000F2EBF029
:10385000A3EAF0A3E9F0E47F08FEFDFC9000EEE0AF
:10386000F8A3E0F9A3E0FAA3E0FB12024CE42FFF77
:10387000E43EFEED3401FDE43CFC9000F2E0FBA3ED
:10388000E0FAA3E0F99000FC7408F0122B77229084
:1038900000A2EEF0A3EFF0A3EDF0A37403F090000C
:1038A000A2E0FEA3E0FFA3E0FB7D42122A7A900093
:1038B000A2E0FEA3E0FF9000E2E4F0A3F0A3F0FB9F
:1038C0007D42121B25EF7002FF229000A5E014F04C
:1038D000E0D3940050C87F01229000A1EFF0047063
:1038E00005E49000A1F09000A1E004F0E4A3F0A3AF
:1038F000F09000A2E0FDC3946050219000A1E0751B
:10390000F080A47C002DFFEC35F0FE1241A8900061
:10391000A3E02FF09000A2E004F080D59000A3E097
:10392000FF2290009FEDF0A3EBF0A3EAF0A3E9F0F3
:10393000123B6590009FE0FF14F0EF6023A3E0FBD3
:10394000A3E475F0011201A6A9F0FA120104FF9098
:1039500000A3F0123E419000A3E02528F52880D373
:10396000AF28123E4112400F229000FD12049A121D
:103970003FC1C2849000FDE0FCA3E0FDA3E0FEA3F4
:10398000E0FF90010712049A7F83121622D28490DE
:1039900000FDE0FCA3E0FDA3E0FEA3E0FF78081239
:1039A0000390EFEEE49001A4EEF0A3EFF022C2D575
:1039B000E830E70FB2D5E4C39BFBE49AFAE499F947
:1039C000E498F8EC30E717B2D51239E41202D7E4E4
:1039D000C39BFBE49AFAE499F9E498F88003120295
:1039E000D730D50DE4C39FFFE49EFEE49DFDE49C2B
:1039F000FC22124180D284C2B7A2B5B392B57F0532
:103A00007E00124086A2B5B392B57F057E001240BB
:103A100086A2B5B392B57F057E00124086A2B5B3EB
:103A200092B57F057E00124086D2B7A2B5B392B59B
:103A3000124180229000BB12049AC003C002C00150
:103A4000E47F08FEFDFC9000BBE0F8A3E0F9A3E0F2
:103A5000FAA3E0FB12024CE42FFFE43EFEED34013A
:103A6000FDE43CFC9000DF7408F0D001D002D003EC
:103A700012361D22E490018EF0A3F0A3F0A3F0A370
:103A8000F0A304F0A3F09000F7F0A37401F0A37486
:103A90008EF0E4FB7D077FA0123BD29000F774010B
:103AA000F0A37401F0A3748EF07B3A7D017FA01225
:103AB0003BD2227B017A0079D31219F19000D9E030
:103AC000FB7A007C007D18FF7E0012017EAA06AB07
:103AD000079000D6E02BFBE43AFA7D3CAF03FE12E0
:103AE000017EAA06AB07A3E02BFBE43AFAFEAF0384
:103AF0002290009FEFF0047005E490009FF090008A
:103B00009FE004F0E4A3F09000A0E0FDD3946050A7
:103B10001B90009FE075F080A47C002DFFEC35F039
:103B2000FE123C069000A0E004F080DB229000F141
:103B3000EBF0A3EAF0A3E9F09000F1E0FBA3E0FAD8
:103B4000A3E0F912302B9000F1E0F9A3E0FAA3E032
:103B50009000F7C9F0A3EAF0A3E9F07B207D0C7F89
:103B6000A0123BD2229000AFEFF0E4FF1240F47FAE
:103B700042123E417F62123E417F13123E4190004D
:103B8000AFE0FF123E41E4F52874A42528F528246F
:103B900013F5289000AFE02528F52822B2B5900053
:103BA0000075F000E49325F0F5F0A3E58270F5E5EB
:103BB00083B2B5B448EE85F01DE51D6014C2A57F43
:103BC000B87E0B123FF5D2A57FB87E0B123FF58071
:103BD000EC22ED6030124149EF54F04402FF123FF5
:103BE0008DAF03123F8D9000F7E0FBA3E475F00169
:103BF0001201A6A9F0FA120104FF123F8DDDE712AF
:103C00004167124028229000A1EEF0A3EFF0123F8E
:103C1000C1C2849000A1E0FEA3E0FFE4FCFD7808AF
:103C20001203A490010712049A7F81121622D284F3
:103C300074FF9001A4F0A3F022900106EFF0900130
:103C400006E0601AC2A57FC87E00124086D2A57F1A
:103C5000C87E00124086900106E014F080E07FD01C
:103C60007E07124086A2B5B392B522ED75F021A46D
:103C7000FF9000D7E07C002FFFEC35F0FEEF7802DC
:103C8000C333CE33CED8F92480FFEE344FFEE4FCAC
:103C9000FD9000DF7404F012361D2290009FEEF0BC
:103CA000A3EFF0A3EDF0E4FB7D45122A7A90009F8C
:103CB000E0FEA3E0FF9000E27401F0A37400F0A323
:103CC00074A2F07B017D45121B252212314EAD07F7
:103CD000AC06D281D3ED9467EC940D40037F0D22A6
:103CE000D3ED941FEC940C40037F0722D3ED942076
:103CF000EC940340037F08227F0D229000A1EEF098
:103D0000A3EFF0AE04AF05E4FCFD78081203A412A3
:103D10002D489000A1E0FEA3E0FFE4FCFD7808122E
:103D200003A4123969229000FD12049A123FC1C205
:103D3000849000FDE0FCA3E0FDA3E0FEA3E0FF9083
:103D4000010712049A7F58121622D284221205C843
:103D500090008FEEF0A3EFF07F011240F490008FFF
:103D6000E0FEA3E0FFF47002EEF46006EF64624E42
:103D700070DB2290008EEFF0123DB97FD07E0712EB
:103D80004086D20590008EE0FF123F39E4FF122DED
:103D9000B8123D4D80FB22C28E53890F43891075A6
:103DA0008BEB758DCBC28FD28E209808308FFAC2E4
:103DB0008E7F0022C28E7F01227E007F0E7D007BDF
:103DC000017A01794C12051E7E007F027DFF7B0186
:103DD0007A01794C12051E123EDF2290009FEFF00F
:103DE0007F2B123B6590009FE0FF123E4190009FA9
:103DF000E02528F528FF123E4112400F2290009F37
:103E0000EFF07F2D123B6590009FE0FF123E419046
:103E1000009FE02528F528FF123E4112400F229016
:103E20000090EFF07F3F123B65900090E0FF123E64
:103E300041900090E02528F528FF123E4112400FE6
:103E400022AD079001A67404F020990B9001A6E022
:103E500070F77EFF7FFF22C299AF058F997E007FAA
:103E6000002290009FEDF0123B6590009FE0FF1252
:103E70003E4190009FE02528F528FF123E41124068
:103E80000F22E49001ABF09001ABE0FFC36480949B
:103E9000A0500B1211619001ABE004F080E97F00AB
:103EA0002290014CE0FF13B3920FEFA2E19223A204
:103EB000E2921CA2E39213A2E49211A2E5920222E2
:103EC000AE04ED7802C333CE33CED8F924E0FFE45C
:103ED0003EFEE4FCFD9000DF7404F012361D221259
:103EE0003EA11235CA9000F77401F0A37401F0A34B
:103EF000744CF07B2C7D0E7FA0123BD2227B017A8A
:103F00000079AC1237FA9000B0E0FCA3E0FDA3E02A
:103F1000FEA3E0FF90018612049A227B017A0079C9
:103F20009F1237FA7B017A00799F12308C7B017ADD
:103F300000799F123B2D7F0022AD07AF051DEF607A
:103F400014C2A57F327E00124086D2A57FC87E00B3
:103F500012408680E622ED25E0FFEC33FEEF246080
:103F6000FFEE3401FEE4FCFD9000DF7402F0123637
:103F70001D220000070001034301000101000000B1
:103F8000000C00040101050000050108007E08EF97
:103F9000339296D297EF25E0FFC297DEF2C29600E9
:103FA000D2970000C29722D2967E08C29712000ACA
:103FB000D297EF25E0FDA296E4334DFFDEEDC297E8
:103FC000221241807DC8124129EFF46004EF20E7FE
:103FD00009DDF37F02123C3980F9227B017A0179F5
:103FE0004C9000F6742CF07D0E7FA0122E27123E0E
:103FF000A112376022AB07AA06EB1BAE0270011AB2
:104000004E600BB2B57F017E0012408680EB22909D
:1040100001A67404F020990B9001A6E070F77EFFD2
:104020007FFF227E007F0022C28E53890F438910BA
:10403000758BEB758DCBC28FD28E308FFDC28E22E9
:10404000C28E53890F438910758BCB758DFAC28F41
:10405000D28E308FFDC28E227F011240F49001A7D4
:104060007401F0123269BEFFFABFFFF77F01226AC6
:1040700050202D20706C204D6F6E61204C69736153
:10408000203230303100EF1FAC0670011ED3940097
:10409000EC64809480400512404080EA22C2AF5315
:1040A00089F0438901758A3E758C5DC2B9D2A9D267
:1040B0008CD2AF227F08E4FEC297EE25E0FE30826C
:1040C000010ED29700DFF1AF06227F011240F4E427
:1040D0009001A7F0123269BEFFFABFFFF77F0122FD
:1040E000EF75F00A84FEC454F0FEEF75F00A84E523
:1040F000F04EFF22EF700BD293C2B67F03FE124048
:104100008622D2B6C293227E08EF339283C297EF03
:1041100025E0FFD297DEF2221201BCFFAEF0900044
:104120000212011DFD123C9B22124180C2847F5766
:104130001241071240B4D284227E007F047D007BAE
:10414000017A01797E12051E22D296D29712000AB8
:1041500000C2960000C29722EFC4540F75F00AA463
:10416000FEEF540F2EFF22C29612000AD2971200C1
:104170000AD296227E007F087D0012051E7F012252
:10418000D2B7D284D283D282D29722E4F518D2A7B2
:10419000D2A5C22522C2AF7F011240F480FE22C206
:1041A00096D2970000C29722E4FD1236C122420146
:1041B000A4FFFF007F0022D28122FFFFFFFFFFFF4D
:1041C000FFFFFFFFFFFFFFFFFFFFFFFFFFFFFFFFFF
:1041D000FFFFFFFFFFFFFFFFFFFFFFFFFFFFFFFFEF
:1041E000FFFFFFFFFFFFFFFFFFFFFFFFFFFFFFFFDF
:1041F000FFFFFFFFFFFFFFFFFFFFFFFFFFFFFFFFCF
:1047F000FFFFFFFFFFFFFFFFFFFFFFFFFFFFFFA721
:00000001FF
